:020000040000FA
:040000003CEF00F0E1
:020008004BD0DB
:0800180099D0036A026EFF0E8D
:100020000226032200D0D8A01200030E016EE70EB4
:1000300002D8F5D7016AFE0F006EE86A015AD8A00F
:1000400012000000000600D0F8D7056A046A100EFE
:10005000F36E0134043605360250045C0350055833
:1000600005E30250045E0350055AD880003601367D
:10007000F32EEFD700501200F86A4F0EAF6E240E29
:10008000AC6E900EAB6E0001C69A540E926EE00EEE
:10009000936EC00E946E070EB46E0F0EC16EA8D094
:1000A0009EAA1BD0060EAB1412E1E1CF23F0E2CFE3
:1000B00024F0252A1EEE80F02550E126000EE222D3
:1000C000AECFE7FF23C0E1FF24C0E2FF1100AE5036
:1000D000AE50AB98AB8811000AD0F2A408D0F294CD
:1000E000084A092A8070076AD6CF06F0110011006D
:1000F0002550265C14E0262AE9CF00F0EACF01F073
:100100000EEE80F02650E926000EEA22EF50006E37
:1001100000C0E9FF01C0EAFFD880120004D0E868FF
:10012000006ED8A012001200256A266A9D8A9F8A56
:10013000F28EF28C12009D9A0EEE80F0000EEE6AA6
:10014000E82EFDD7256A266A9D8A1200F29ED8CF36
:100150005AFEE8CF5BFEE0CF5CFEE9CF5DFEEACF62
:100160005EFEE1CF5FFEE2CF60FED9CF61FEDACF67
:1001700062FEF6CF63FEF7CF64FEF5CF65FEF3CFE8
:1001800066FEF4CF67FEA6CF68FEF28E0001A19254
:10019000B90EB26EB30EB36E202A400E205C03E19E
:1001A0001C4A1D2A206AF29E5ACED8FF5BCEE8FF79
:1001B0005CCEE0FF5DCEE9FF5ECEEAFF5FCEE1FF01
:1001C00060CEE2FF61CED9FF62CEDAFF63CEF6FFEA
:1001D00064CEF7FF65CEF5FF66CEF3FF67CEF4FF82
:1001E00068CEA6FFF28E10009EA8FED7AD6E12005C
:1001F00094988B9894968B9693908A9093928A92E7
:1002000093948A9493968A9693988A98949A8B9AC0
:1002100092928992929A899A9296899694948B94C2
:10022000196A166A216A92908980320EF6DE9290DF
:1002300089907ADF80DFCD6AF294F28A870ED56EDC
:10024000B16AA192A082B26AB36AD08EA292B10EB4
:10025000B16E4EDF0A6EC10E0A5C07E3FE0E0A5C49
:1002600002E3F7D702D00C6AF4D70AAE2DD00C6A9D
:100270008992800E0A5C06E10AC00CF00D680E68D7
:10028000898221D0900E0A5C06E10AC00CF00F684A
:100290001068898218D0A00E0A5C06E10AC00CF032
:1002A0001168126889820FD0B00E0A5C05E10AC09D
:1002B0000CF01368146807D0C00E0A5C04E10AC091
:1002C0000CF01668898254D10C5203E18992C1D78F
:1002D0004FD1800E0C5C16E10D2803E10AC00DF031
:1002E00010D00AC00EF0020E0D5C09E18B988B96BF
:1002F0008A908A928A948A968A988B9A01D0899257
:100300000D6836D1900E0C5CD8A4CDD00F2803E137
:100310000AC00FF0C7D00AC010F0020E0F5CD8A4BC
:10032000BFD010BA828A10AA829A109A105208E19D
:100330008B888B868A808A828A848A868A98AFD0C4
:10034000010E105C08E18B988B868A808A928A94D1
:100350008A968A98A4D0020E105C08E18B888B865E
:100360008A888A848A828A908A9699D0030E105C41
:1003700008E18B888B868A808A828A948A968A880A
:100380008ED0040E105C08E18B988B868A808A924E
:100390008A948A868A8883D0050E105C08E18B884F
:1003A0008B968A808A828A948A868A8878D0060E7A
:1003B000105C08E18B888B968A808A828A848A8680
:1003C0008A886DD0070E105C08E18B888B868A8046
:1003D0008A928A948A968A9862D0080E105C08E104
:1003E0008B888B868A808A828A848A868A8857D07C
:1003F000090E105C08E18B888B868A808A828A9439
:100400008A868A884CD00A0E105C08E18B888B861D
:100410008A808A928A848A868A8841D00B0E105CF0
:1004200008E18B988B968A808A828A848A868A8859
:1004300036D00C0E105C08E18B888B968A908A82ED
:100440008A848A868A982BD00D0E105C08E18B98DE
:100450008B868A808A828A848A968A8820D00E0E29
:10046000105C08E18B888B968A908A828A848A86BF
:100470008A8815D00F0E105C08E18B888B968A90C5
:100480008A928A848A868A880AD0100E105C07E1D4
:100490008B988B968A908A928A948A968A9801D0B1
:1004A00089920F6865D0A00E0C5C2AE1112803E147
:1004B0000AC011F024D00AC012F0020E115C1DE136
:1004C00012B0818812A0819812B2818612A2819600
:1004D00012B4818412A4819412B6818212A68192F0
:1004E00012B8818012A8819012BA828612AA8296CE
:1004F00012BC828812AC829801D08992116838D0DF
:10050000B00E0C5C0AE1132803E10AC013F004D01A
:100510000AC014F07CEC05F02BD0C00E0C5C28E176
:100520000CC015F0162824E10AC016F0A5EC05F061
:10053000215202E18ED61CD0010E215C02E119D0BD
:1005400017D0020E215C03E111EF06F011D0030E6B
:10055000215C03E185EF07F00BD0040E215C03E181
:10056000C5EF08F005D0050E215CD8B425EF0AF0E0
:1005700070D678EC00F00A6EC10E0A5C07E3FE0E3E
:100580000A5C02E3F6D702D00C6AF3D70AAE2FD08A
:100590000C6A8992800E0A5C06E10AC00CF00D68B4
:1005A0000E68898222D0900E0A5C06E10AC00CF027
:1005B0000F681068898219D0A00E0A5C06E10AC093
:1005C0000CF011681268898210D0B00E0A5C06E146
:1005D0000AC00CF013681468898207D0C00E0A5C48
:1005E00004E10AC00CF0166889827AEF05F00C521B
:1005F00003E189927AEF05F0800E0C5C18E10D287A
:1006000003E10AC00DF011D00AC00EF0020E0D5C1D
:100610000AE18B988B968A908A928A948A968A9815
:100620008B9A8B9401D089920D687AEF05F0900E29
:100630000C5CD8A4FDD10F2803E10AC00FF0F7D15C
:100640000AC010F0020E0F5CD8A4EFD18B988B96E5
:100650008A908A928A948A968A988B9A8B94070EAB
:10066000105C02E18B84E0D1270E105C02E18B86E6
:10067000DBD12D0E105C02E18A88D6D12E0E105CE3
:1006800002E18B8AD1D12F0E105C04E18B868A8423
:100690008A88CAD1300E105C07E18B888B868A80ED
:1006A0008A828A848A86C0D1310E105C03E18B86EF
:1006B0008A80BAD1320E105C06E18B888B868A88DC
:1006C0008A848A82B1D1330E105C06E18B888B86D6
:1006D0008A808A828A88A8D1340E105C05E18B86D4
:1006E0008A808A868A88A0D1350E105C06E18B88C4
:1006F0008A808A828A868A8897D1360E105C07E1C2
:100700008B888A808A828A848A868A888DD1370EED
:10071000105C04E18B888B868A8086D1380E105C51
:1007200008E18B888B868A808A828A848A868A8876
:100730007BD1390E105C07E18B888B868A808A8298
:100740008A868A8871D13A0E105C07E18B888B8685
:100750008A808A848A868A8867D13B0E105C06E18B
:100760008A808A828A848A868A885ED13C0E105C5E
:1007700005E18B888A828A848A8656D13D0E105C78
:1007800006E18B868A808A828A848A884DD13E0ED1
:10079000105C06E18B888A828A848A868A8844D1A2
:1007A0003F0E105C05E18B888A848A868A883CD15A
:1007B000410E105C03E0610E105C07E18B888B86B4
:1007C0008A808A828A848A882FD1420E105C03E054
:1007D000620E105C06E18A808A828A848A868A8810
:1007E00023D1430E105C03E0630E105C04E18A82A7
:1007F0008A848A8819D1440E105C03E0640E105C70
:1008000006E18B868A808A828A848A880DD1450E89
:10081000105C03E0650E105C06E18B888A828A8496
:100820008A868A8801D1460E105C03E0660E105C51
:1008300005E18B888A848A868A88F6D0470E105C08
:1008400003E0670E105C06E18B888A808A828A84C6
:100850008A86EAD0480E105C03E0680E105C05E161
:100860008A808A848A868A88DFD0490E105C03E0F9
:10087000690E105C02E18A80D7D04A0E105C03E05A
:100880006A0E105C04E18B868A808A82CDD04B0E82
:10089000105C03E06B0E105C04E18A848A868A880F
:1008A000C3D04C0E105C03E06C0E105C05E18A8234
:1008B0008A848A868A98B8D04D0E105C03E06D0E4B
:1008C000105C05E18B888A808A848A88ADD04E0EC0
:1008D000105C03E06E0E105C04E18A808A848A88D2
:1008E000A3D04F0E105C03E06F0E105C05E18A8010
:1008F0008A828A848A8898D0500E105C03E0700E39
:10090000105C06E18B888B868A848A868A888CD0E4
:10091000510E105C03E0710E105C06E18B888B8633
:100920008A808A868A8880D0520E105C03E0720E1C
:10093000105C03E18A848A8877D0530E105C03E050
:10094000730E105C05E18B888A808A828A866CD05F
:10095000540E105C03E0740E105C05E18A828A84F8
:100960008A868A8861D0550E105C03E0750E105C93
:1009700004E18A808A828A8457D0560E105C03E094
:10098000760E105C05E18B868A808A848A864CD03C
:10099000570E105C03E0770E105C05E18B868A82AF
:1009A0008A868A8841D0580E105C03E0780E105C6D
:1009B00004E18B888A828A8837D0590E105C03E064
:1009C000790E105C06E18B868A808A828A868A8804
:1009D0002BD05A0E105C03E07A0E105C05E18B8878
:1009E0008B868A828A8420D05C0E105C04E18A8027
:1009F0008A868A8819D05D0E105C05E18B888B860B
:100A00008A808A8211D05E0E105C04E18B888B860E
:100A10008A860AD05F0E105C02E18A8205D07C0EC5
:100A2000105C02E18A848A8601D089920F6862D0C4
:100A3000A00E0C5C2AE1112803E10AC011F024D0B9
:100A40000AC012F0020E115C1DE112B0818812A0E2
:100A5000819812B2818612A2819612B4818412A466
:100A6000819412B6818212A6819212B8818012A856
:100A7000819012BA828612AA829612BC828812AC27
:100A8000829801D08992116835D0B00E0C5C09E1D2
:100A9000132803E10AC013F003D00AC014F02CD8C5
:100AA00029D0C00E0C5C26E1162824E10AC016F0FD
:100AB0004CD8215203E129EF01F01CD0010E215C3A
:100AC00003E1B9EF02F016D0020E215C02E1A9D0D9
:100AD00011D0030E215C03E185EF07F00BD0040E6B
:100AE000215C03E1C5EF08F005D0050E215CD8B408
:100AF00025EF0AF0B9EF02F01A0E135C07E173D884
:100B0000020E215C02E11A6A1B6A1CD01B0E135CE8
:100B100007E1020E215C03E102D01A4A1B2A12D01F
:100B2000420E135C0BE1145205E11A6A1B6A19901C
:100B30006BD803D01A6A1B6A198004D07B0E135C31
:100B4000D8B451D8899213681200165204E115687E
:100B500016C021F044D0010E165C04E1156816C0E1
:100B600021F03DD0020E165C09E13DD815681A6AE5
:100B70001B6A1E6A1F6A16C021F031D0030E165C74
:100B80000BE131D81568206A1C6A1D6A1E6A1F6A4B
:100B90008B9A16C021F023D0040E165C14E18B88CA
:100BA0008B868A808A828A848A868A98899A8B8AA6
:100BB00001D08B9A1568206A1C6A1D6A1E6A1F6A1A
:100BC00016C021F00CD0050E165C09E11568206AEC
:100BD0001C6A1D6A1E6A1F6A8B9A16C021F00C6877
:100BE0008992166812008B988B968A908A928A94C2
:100BF0008A968A988B9A899A89961A6A1B6A206AB9
:100C00001C6A1D6A8B9412008B988B968A908A922C
:100C10008A948A968A988B9A8992899A89968B94D3
:100C2000120078EC00F00A6EC10E0A5C07E3FE0EBB
:100C30000A5C02E3F6D702D00C6AF3D70AAE2DD0D5
:100C40000C6A8992800E0A5C06E10AC00CF00D68FD
:100C50000E68898221D0900E0A5C06E10AC00CF071
:100C60000F681068898218D0A00E0A5C06E10AC0DD
:100C70000CF01168126889820FD0B00E0A5C05E191
:100C80000AC00CF01368146807D0C00E0A5C04E1B7
:100C90000AC00CF0166889826CD00C5202E189926D
:100CA00068D0800E0C5C0AE10D2803E10AC00DF04B
:100CB00004D00AC00EF00D6889925BD0900E0C5CD7
:100CC00016E10F2803E10AC00FF010D00AC010F09F
:100CD00010C000F0016A0A0E026E036A25EC00F0F3
:100CE00004C01AF005C01BF00F68899242D0A00E14
:100CF0000C5C0AE1112803E10AC011F004D00AC01B
:100D000012F01168899235D0B00E0C5C09E11328FD
:100D100003E10AC013F003D00AC014F0EDDE29D0BD
:100D2000C00E0C5C26E10CC015F0162822E10AC0AA
:100D300016F00BDF215203E129EF01F01AD0010E6A
:100D4000215C03E1B9EF02F014D0020E215C02E154
:100D500068D70FD0030E215C02E1D7D00AD0040E71
:100D6000215C02E112D205D0050E215CD8B425EF3A
:100D70000AF080B4899A21D080A806D080B603D02A
:100D80001A4A1B2A898601D089961AC000F01BC016
:100D900001F00A0E026E036A25EC00F004C01EF09A
:100DA0001E50225C09E01A5202E11B5203E01E525F
:100DB000D8B4898A1EC022F03BD001D021D080A8AF
:100DC00006D080B603D01A4A1B2A898601D089969C
:100DD0001AC000F01BC001F00A0E026E036A25EC77
:100DE00000F004C01EF01E50225C09E01A5202E11D
:100DF0001B5203E01E52D8B4898A1EC022F018D0BC
:100E000017D01AC000F01BC001F00A0E026E036A70
:100E100025EC00F004C01EF01E50225C09E01A52BE
:100E200002E11B5203E01E52D8B4898A1EC022F090
:100E30001E5208E18B888B868A808A828A848A8601
:100E40008A9862D0010E1E5C08E18B988B868A809E
:100E50008A928A948A968A9857D0020E1E5C08E17C
:100E60008B888B868A888A848A828A908A964CD0DC
:100E7000030E1E5C08E18B888B868A808A828A94A6
:100E80008A968A8841D0040E1E5C08E18B988B8676
:100E90008A808A928A948A868A8836D0050E1E5C59
:100EA00008E18B888B968A808A828A948A868A88CF
:100EB0002BD0060E1E5C08E18B888B968A808A8276
:100EC0008A848A868A8820D0070E1E5C08E18B8877
:100ED0008B868A808A928A948A968A9815D0080E80
:100EE0001E5C08E18B888B868A808A828A848A8647
:100EF0008A880AD0090E1E5C07E18B888B868A805F
:100F00008A828A948A868A888CD678EC00F00A6E67
:100F1000C10E0A5C07E3FE0E0A5C02E36AD002D04F
:100F20000C6A67D00AAE29D00C6A8072800E0A5C07
:100F300005E10AC00CF00D680E681ED0900E0A5C28
:100F400005E10AC00CF00F68106816D0A00E0A5C0C
:100F500005E10AC00CF0116812680ED0B00E0A5CF0
:100F600005E10AC00CF01368146806D0C00E0A5CD4
:100F700003E10AC00CF016683CD0A10E0C5C02E242
:100F800038D037D0B00E0C5C0AE1132803E10AC058
:100F900013F004D00AC014F07CEC05F02AD0C00E87
:100FA0000C5C27E10CC015F0162823E10AC016F0EE
:100FB000A5EC05F0215203E129EF01F01AD0010E52
:100FC000215C03E1B9EF02F014D0020E215C02E1D2
:100FD00028D60FD0030E215C02E197D70AD0040E69
:100FE000215C02E1D2D005D0050E215CD8B425EFFA
:100FF0000AF080B4899A21D080A806D080B603D0A8
:101000001A4A1B2A898601D089961AC000F01BC093
:1010100001F00A0E026E036A25EC00F004C01EF017
:101020001E50225C09E01A5202E11B5203E01E52DC
:10103000D8B4898A1EC022F03BD001D021D080A82C
:1010400006D080B603D01A4A1B2A898601D0899619
:101050001AC000F01BC001F00A0E026E036A25ECF4
:1010600000F004C01EF01E50225C09E01A5202E19A
:101070001B5203E01E52D8B4898A1EC022F018D039
:1010800017D01CC000F01DC001F00A0E026E036AEA
:1010900025EC00F004C01EF01E50225C09E01C523A
:1010A00002E11D5203E01E52D8B4898A1EC022F00C
:1010B0001E5208E18B888B868A808A828A848A867F
:1010C0008A9862D0010E1E5C08E18B988B868A801C
:1010D0008A928A948A968A9857D0020E1E5C08E1FA
:1010E0008B888B868A888A848A828A908A964CD05A
:1010F000030E1E5C08E18B888B868A808A828A9424
:101100008A968A8841D0040E1E5C08E18B988B86F3
:101110008A808A928A948A868A8836D0050E1E5CD6
:1011200008E18B888B968A808A828A948A868A884C
:101130002BD0060E1E5C08E18B888B968A808A82F3
:101140008A848A868A8820D0070E1E5C08E18B88F4
:101150008B868A808A928A948A968A9815D0080EFD
:101160001E5C08E18B888B868A808A828A848A86C4
:101170008A880AD0090E1E5C07E18B888B868A80DC
:101180008A828A948A868A88C0D678EC00F00A6EB1
:10119000C10E0A5C07E3FE0E0A5C02E36AD002D0CD
:1011A0000C6A67D00AAE29D00C6A8072800E0A5C85
:1011B00005E10AC00CF00D680E681ED0900E0A5CA6
:1011C00005E10AC00CF00F68106816D0A00E0A5C8A
:1011D00005E10AC00CF0116812680ED0B00E0A5C6E
:1011E00005E10AC00CF01368146806D0C00E0A5C52
:1011F00003E10AC00CF016683CD0A10E0C5C02E2C0
:1012000038D037D0B00E0C5C0AE1132803E10AC0D5
:1012100013F004D00AC014F07CEC05F02AD0C00E04
:101220000C5C27E10CC015F0162823E10AC016F06B
:10123000A5EC05F0215203E129EF01F01AD0010ECF
:10124000215C03E1B9EF02F014D0020E215C03E14E
:1012500011EF06F00ED0030E215C02E156D609D044
:10126000040E215C02E191D704D0050E215CD8B4B4
:10127000ECD080B4899A21D080A806D080B603D063
:101280001A4A1B2A898601D089961AC000F01BC011
:1012900001F0060E026E036A25EC00F004C01EF099
:1012A0001E50225C09E01A5202E11B5203E01E525A
:1012B000D8B4898A1EC022F05BD080A806D080B640
:1012C00003D01A4A1B2A898601D089961AC000F0D9
:1012D0001BC001F00A0E026E036A25EC00F004C088
:1012E0001EF01E50225C09E01A5202E11B5203E07C
:1012F0001E52D8B4898A1EC022F03AD021D080A8CC
:1013000006D080B603D01A4A1B2A898601D0899656
:101310001AC000F01BC001F0060E026E036A25EC35
:1013200000F004C01EF01E50225C09E01A5202E1D7
:101330001B5203E01E52D8B4898A1EC022F018D076
:1013400017D01CC000F01DC001F00A0E026E036A27
:1013500025EC00F004C01EF01E50225C09E01C5277
:1013600002E11D5203E01E52D8B4898A1EC022F049
:101370001E5208E18B888B868A808A828A848A86BC
:101380008A9862D0010E1E5C08E18B988B868A8059
:101390008A928A948A968A9857D0020E1E5C08E137
:1013A0008B888B868A888A848A828A908A964CD097
:1013B000030E1E5C08E18B888B868A808A828A9461
:1013C0008A968A8841D0040E1E5C08E18B988B8631
:1013D0008A808A928A948A868A8836D0050E1E5C14
:1013E00008E18B888B968A808A828A948A868A888A
:1013F0002BD0060E1E5C08E18B888B968A808A8231
:101400008A848A868A8820D0070E1E5C08E18B8831
:101410008B868A808A928A948A968A9815D0080E3A
:101420001E5C08E18B888B868A808A828A848A8601
:101430008A880AD0090E1E5C07E18B888B868A8019
:101440008A828A948A868A88A0D678EC00F00A6E0E
:10145000C10E0A5C07E3FE0E0A5C02E3F6D702D077
:101460000C6AF3D70AAE2DD00C6A8992800E0A5C02
:1014700006E10AC00CF00D680E68898221D0900E3A
:101480000A5C06E10AC00CF00F681068898218D067
:10149000A00E0A5C06E10AC00CF01168126889828D
:1014A0000FD0B00E0A5C05E10AC00CF01368146896
:1014B00007D0C00E0A5C04E10AC00CF016688982ED
:1014C00082D1800E0C5C09E10D2803E10AC00DF009
:1014D00003D00AC00EF00D6876D1900E0C5CD8A433
:1014E00013D10F2803E10AC00FF00DD10AC010F08C
:1014F000050E0F5CD8B006D18B988B968A908A9295
:101500008A948A968A988B9A02D09294899451D020
:101510001052D8B44DD0010E105C03E1929489842E
:1015200047D0020E105C04E1929489848A8240D0F4
:10153000030E105C04E1929489848A8439D0040EED
:10154000105C05E1929489848A848A8831D0050EE2
:10155000105C05E1929489848A848A8629D0060EDB
:10156000105C06E1929489848B888A848A8620D0D4
:10157000070E105C07E1929489848B888B868A849D
:101580008A8616D0080E105C08E1929489848B88B4
:101590008B868A808A848A860BD0090E105C08E3C9
:1015A000929489848B888B868A808A848A868B8AA7
:1015B000A9D00A0E105C02E18A8232D00B0E105CB8
:1015C00002E18A842DD00C0E105C03E18A848A88A3
:1015D00027D00D0E105C03E18A848A8621D00E0E7E
:1015E000105C04E18B888A848A861AD00F0E105C06
:1015F00005E18B888B868A848A8612D0100E105C57
:1016000006E18B888B868A808A848A8609D0110EAF
:10161000105C06E38B888B868A808A848A868B8A14
:1016200071D038D0120E105C02E18A8232D0130ED3
:10163000105C02E18A842DD0140E105C03E18A84D0
:101640008A8827D0150E105C03E18A848A8621D00F
:10165000160E105C04E18B888A848A861AD0170ED5
:10166000105C05E18B888B868A848A8612D0180EDE
:10167000105C06E18B888B868A808A848A8609D0F2
:10168000190E105C06E38B888B868A808A848A8692
:101690008B8A38D037D01A0E105C02E18A8232D0A1
:1016A0001B0E105C02E18A842DD01C0E105C03E13D
:1016B0008A848A8827D01D0E105C03E18A848A867A
:1016C00021D01E0E105C04E18B888A848A861AD091
:1016D0001F0E105C05E18B888B868A848A8612D067
:1016E000200E105C06E18B888B868A808A848A862D
:1016F00009D0210E105C06E38B888B868A808A8451
:101700008A868B8A0F685FD0A00E0C5C09E11128D5
:1017100003E10AC011F003D00AC012F0116853D0DF
:10172000B00E0C5C0AE1132803E10AC013F004D0E8
:101730000AC014F07CEC05F046D0C00E0C5CD8A4B6
:1017400042D00CC015F016283EE10AC016F0A5ECF8
:1017500005F0215208E102D092948994540E926EC1
:1017600029EF01F030D0010E215C08E102D0929403
:101770008994540E926EB9EF02F025D0020E215CCE
:1017800008E102D092948994540E926E11EF06F003
:101790001AD0030E215C08E102D092948994540E71
:1017A000926E85EF07F00FD0040E215C08E102D0A5
:1017B00092948994540E926EC5EF08F004D0050EF1
:0A17C000215CD8B442D641D6FFD711
:020000040030CA
:0300010006170ED1
:020005008580F4
:060008000FC00FE00F40E5
:00000001FF
